:020000040000FA
:100000002E2882073F34D53416348334013490349B
:10001000303480340034813430343F34003485341B
:1000200001349F341234833430340734003499342B
:100030000134A0341C34053428340B340A34A03481
:10004000163483340834203400349034123483342A
:10005000183405342834123428340B348316FF2323
:100060009000A03081000E3085009F018312073080
:10007000990010308500872108308B0083160830E6
:1000800096008312630000006F2061204C208B20BB
:10009000851205162C213C281B2122217A217A2148
:1000A0001530A4000130AC00AC0A2C080120A700D8
:1000B000AC0A2C080120A800D6200321A40B542848
:1000C00008001B2122217A217A2113210B210B21E7
:1000D00013210B210B218721872187210800003064
:1000E0000120A20001300120A3001B212221831640
:1000F000851083129E200321032103210321032164
:1001000003210321AD2030302705A600CF30220582
:100110002604A20008001B212221831685108312C9
:100120009E20032103210321032103210321032115
:100130002308A8002208A700D62008000B210B21C5
:100140000B210B210B210B211030A4000514000002
:1001500000000510A40BA628080083168510831242
:100160000B210B2113210B210B210B21831685144D
:1001700083120830AD000514051000000514A80C0A
:10018000A817851CA8130510AD0BBE280630AD00BE
:100190000514A70CA716851CA7120510AD0BC828BF
:1001A0003F30A705051405100000080083168510D0
:1001B00083120B2113210B210B210B210B21083062
:1001C000AD0005148510051005148514281C851034
:1001D0000510A80CAD0BE4280630AD0005148514FD
:1001E000271C85100510A70CAD0BEE2805148510F3
:1001F00005107A210B210B210B2113210B210B213F
:100200008721872108000B21132113210B210B21AA
:100210000B217A2108000514000000008510000061
:1002200000000510080005140000000085140000FF
:10023000000005100800851205168121831685141B
:100240008312080083168510831285100510851609
:100250007A2105127A21080087218721051287213A
:10026000831685108312AE01FF30A40085147A2115
:100270007A21851081218121812181016330AD00A6
:100280000000AD0B4029000000000108A600AE0AE6
:10029000C730260603195A29C830260603195A29D9
:1002A000C930260603195A29A40B362961208B2050
:1002B0000516080061201B2122217A217A210830AD
:1002C000A4007F30AD000321AD0B63297F30AD006A
:1002D000A40B63290321032103210321032103210B
:1002E00003213430A7002E08A800D6208B20051645
:1002F000851208000000000000000000000000005F
:100300000800FF30A900AA000230AB008D29FF30A1
:10031000A9000830AA000130AB00A90B8D29AA0B57
:080320008D29AB0B8D290800AB
:02400E00D43F9D
:00000001FF
